:020000040000FA
:020000001228C4
:08000800BA00030E8301BB00E6
:100010000A08BC003C088A003B0E8300BA0E3A0E68
:100020000C1009008316FF30850000308600013077
:100030008700811384309F008312C6308700D70168
:10004000D601EB01EC018A154D268A110E24861784
:10005000851A2F28D623F6235714851E2D28051A16
:100060003628D623F623D717051E342805193B2832
:10007000D623F623372604303524EA000030352411
:10008000E90002303524E80014303524E000103057
:100090003524DF000C303524DE0057185428D71BD8
:1000A0005428051A5528561456285610D71B0425CF
:1000B000571859245618E225EC0F6328EB0A033031
:1000C0006B0203198613F623F623F62356186D28C0
:1000D00057186D28D71B6D28051970288A15002818
:1000E000D63087008316213087008312E8238630BC
:1000F00087004D23D63087003E08DA003D08DB003C
:1001000003305A0203198A288316013087008312AC
:10011000F623BA283D245A08A1005B08A000073046
:10012000A40049244D2429243124292420302124C9
:1001300053302124633021243408303E21243508F3
:10014000303E21243608303E2124013021242D2444
:1001500031242D2443302124783021242D302124B2
:1001600073302124633021242D3021242030212498
:100170005D234D28EB01EC01D6308700E8234630A3
:1001800087004D23D63087003E08D8003D08D900AF
:10019000E823463087000630BE00BE0BCD280000A5
:1001A0004D23D63087003E08DA003D08DB000330DF
:1001B0005A0203191F293D245A08A1005B08A00018
:1001C0005808A5005908A4004524A308031D3D2490
:1001D00041242108A5002008A4005808A1005908BE
:1001E000A0004524A308031D3D24412408303524E4
:1001F000A4004524A308031D3D242108D3002008A2
:10020000D2003D240330A5006930A4005E08A000A0
:10021000552441245308A5005208A4005124412428
:100220000130A5005530A40049242108DC00200835
:10023000DD005717D712571256184D28342A831647
:10024000213087008312ED23463087004D23D630BE
:1002500087003E08D8003D08D900E82346308700D3
:100260000630BE00BE0B322900004D23D630870079
:100270003E08DA003D08DB00831601308700831258
:1002800003305A02031978293D245A08A1005B085B
:10029000A0005808A5005908A4004524A308031D80
:1002A0003D2441246630A40051242108D3002008B5
:1002B000D2003D245808A1005908A0005F08A400FE
:1002C000512441245308A5005208A4004524A30842
:1002D000031D3D2441242530A40049242108DC00CD
:1002E0002008DD005713D716571256184D28E42959
:1002F0008316213087008312E823863087004D2340
:10030000D63087003E08D8003D08D900E823863063
:1003100087000230BE00BE0B8B29000000004D2379
:10032000D63087003E08DA003D08DB008316013036
:100330008700831203305A020319D2293D245A0838
:10034000A1005B08A0005808A5005908A400452496
:10035000A308031D3D244124D230A40051242108C8
:10036000D3002008D2003D245808A1005908A0005D
:100370006008A400512441245308A5005208A40099
:100380004524A308031D3D2441244730A4004924EB
:100390002108DC002008DD005713D7125716561825
:1003A0004D280F2A292431242924203021244530A6
:1003B000212473302124723021242D3021242D302A
:1003C00021242D3021240F2A3D245A08A1005B0846
:1003D000A0005808A5005908A40045242108D3000E
:1003E0002008D20041243230A4004524A308031D74
:1003F000342A3D240430A1006030A0006908A40024
:10040000552441243630A400512441245308A5002A
:100410005208A4004924D7105715D711D32A3D24D8
:100420005A08A1005B08A0005808A5005908A400BC
:1004300045242108D3002008D20041240530A4001F
:100440004524A308031DBD2A3D243230A0006A08BC
:10045000A400512441245308A5005208A4004924B3
:10046000D7105711D715D32A1430E7000130E50013
:10047000E6018316213087008312E8234630870087
:100480004D233E08E1003D08E20000004E2A000036
:10049000000000000000000000000000000000005C
:1004A000000000000000000000000000000000004C
:1004B00000000000000000004D2302303E0203183F
:1004C000722AE50F472AE60A3E086102031D4D2AFB
:1004D00062083D02BF0002303F02031CBD2AE70B49
:1004E000552ABD2AD63087003E08E3003D08E400C7
:1004F00083160130870083123D240A30A00068086B
:10050000A400512441241030A500DE30A40055245D
:1005100041246508A4006608A50051242308D500DD
:100520002208D4002108D3002008D2003D2463080B
:10053000A1006408A0006108A5006208A400452489
:100540002108BE002008BD0041240530A400452438
:10055000A308031DBD2A3D243E08A5003D08A400B4
:100560005508A3005408A2005308A1005208A00097
:100570004924D7145711D711D32AD63087008316B0
:100580000130870083122D2431242D24433021246F
:10059000783021242D3021246E3021246F30212405
:1005A000561BAD231D2B4D242D2431242D2420300A
:1005B0002124D71C052B013032020318E82A013010
:1005C00033020318EB2A013034020318F02AF62A0A
:1005D0003208303E21243308303E212420302124AB
:1005E0003408303E2124B208031D002B3508303E6C
:1005F0002124B308031D022B3608303E2124042B8E
:100600003030212430302124192BB30803190B2B4F
:100610003308303E21243408303E21242E3021245A
:100620003508303E2124B308031D192B3608303E0F
:10063000212402302124463021243D245C08A100DD
:100640005D08A0004D2429243124292420302124B0
:10065000571B2D2BB3080319302B3308303E2124B0
:10066000571F342B2C3021243408303E2124D71E30
:100670003B2B2C3021243508303E2124571E422BA1
:100680002C302124D71E472BB308031D4A2B3608D4
:10069000303E2124013021244D2881309F00053037
:1006A000BE00BE0B512B1F151F19542B1E08BE0078
:1006B00083161E088312BD0008003D2489309F0068
:1006C0000530BE00BE0B622B1F151F19652B1E08BF
:1006D000D30083161E088312D2005308A1005208CB
:1006E000A000C730252402302102031D7A2B0330DD
:1006F0002124AC2B3D245308A1005208A000013056
:10070000A500E330A4004524A308031D8A2B043070
:100710002124AC2B3D245308A1005208A000013035
:10072000A500C730A4004524A308031D9A2B05305B
:100730002124AC2B3D245308A1005208A000013015
:10074000A500AB30A4004524A308031DAA2B063046
:100750002124AC2B0730212408003D245808A10097
:100760005908A00008303524A4004524A308031D1F
:100770003D242108D3002008D2003D240330A500E9
:100780006930A4005E08A000552441245308A50048
:100790005208A400512441240130A5005530A40082
:1007A00049242108DC002008DD000800292420302D
:1007B00021245330212465302124723021247630C5
:1007C000212469302124633021246530212408004C
:1007D000FF30BE00BE0BEA2B0800ED30BE004130FA
:1007E000BF00BE0BF12BBF0BF12B0800DC30BE00AD
:1007F0008230BF00BE0BFA2BBF0BFA2B00000800A3
:10080000AC30BE001330BF000630C000BE0B062C5B
:10081000BF0B062CC00B062C0000080048308A15C0
:1008200086268A1107308A003830C2000030C300A3
:1008300000278A156B268A11C30A4308C20B182C9D
:1008400008008A156B268A1108008A1586268A11E7
:1008500008008A159D268A1108008A15A2268A1189
:1008600008008A15AC268A1108008A1560248A11AE
:1008700008008A156B248A1108008A15F4248A114D
:1008800008008A15EF248A1108008A1501258A11AB
:1008900008008A1525258A1108008A15B6258A11AF
:1008A00008008A150E258A1108008A1504258A1168
:1008B0000800D7195F2C5719962CD718CD2C051A7C
:1008C000622CEA0A851A652CEA03292431246A0875
:1008D000A0007F30A40045244D2429242030212469
:1008E00031302124753021243E3021242C1C7A2CD7
:1008F0002D3021243408303E21243508303E212477
:100900003608303E21243C30212420302124051992
:10091000952C2924312429248A15BB248A116A089C
:10092000BD0004303924051D932C0800051A992CAC
:10093000E90A851A9C2CE903292431246908A000BE
:100940007F30A40045244D2429242030212439302F
:100950002124753021243E3021242C1CB12C2D3033
:1009600021243408303E21243508303E2124360825
:10097000303E21243C302124203021240519CC2C68
:100980002924312429248A15BB248A116908BD0031
:1009900000303924051DCA2C0800051AD02CE80A9D
:1009A000851AD32CE803292431246808A0007F305D
:1009B000A40045244D242924203021243930212429
:1009C000753021243E3021242C1CE82C2D3021248C
:1009D0003408303E21243508303E21243608303E8C
:1009E00021243C302124203021240519032D2924E1
:1009F000312429248A15BB248A116808BD000230DD
:100A00003924051D012D0800571B0A2DD71A422D28
:100A1000571A7A2D051A0D2DDE0A851A102DDE03C0
:100A2000292431245E08A0007F30A40045244D24F1
:100A300029242030212431302124523021243E30F9
:100A400021242C1C252D2D3021243408303E212436
:100A50003508303E21243608303E21243C30212404
:100A6000203021240519402D2924312429248A15D8
:100A7000BB248A115E08BD000C303924051D3E2DB3
:100A8000B2250800051A452DDF0A851A482DDF0317
:100A9000292431245F08A0006430A40045244D249B
:100AA0002924203021243130212430302124523097
:100AB00021242C1C5D2D2D3021243408303E21248E
:100AC0003508303E21243608303E21243C30212494
:100AD000203021240519782D2924312429248A1530
:100AE000BB248A115F08BD0010303924051D762D06
:100AF000B2250800051A7D2DE00A851A802DE00335
:100B0000292431246008A0006430A40045244D2429
:100B10002924203021243430212430302124523023
:100B200021242C1C952D2D3021243408303E2124E5
:100B30003508303E21243608303E21243C30212423
:100B4000203021240519B02D2924312429248A1587
:100B5000BB248A116008BD0014303924051DAE2D58
:100B6000B22508003D245C08A1005D08A0004D24CA
:100B70002D2431242D2420302124571BC22DB308CD
:100B80000319C52D3308303E2124571FC92D2C30A1
:100B900021243408303E2124D71ED02D2C3021248E
:100BA0003508303E2124571ED72D2C302124D71E46
:100BB000DC2DB308031DDF2D3608303E2124013023
:100BC000212408005808A1005908A0004D24292418
:100BD00031242924203021243408303E21243508B2
:100BE000303E21243608303E2124571FF92D2B306A
:100BF0002124D71EFD2D2F302124571E012E2D30EC
:100C000021245A08A1005B08A0004D243408303E7E
:100C100021243508303E21243608303E21243D244D
:100C200008303524A0004D242D2431242D242030DB
:100C3000212445302124453021242D30212434081D
:100C4000303E21243508303E21243608303E212410
:100C50000519362E2924312429248A15BB248A110A
:100C60005908BD0008303924051D342E08004030D5
:100C700087002924312429242030212449302124AB
:100C80003D30212431302124303021246D30212485
:100C900041302124F623051A372E8030870029247D
:100CA0003124292420302124493021243D3021249D
:100CB00032302124203021246D3021244130212460
:100CC0000024051E662E851E372E4D2E40308700CF
:100CD0002924312429242030212473302124653013
:100CE00021246B30212431302124303021246D30F7
:100CF000212441302124002450308700292431242C
:100D000029242030212473302124653021246B30A4
:100D1000212420302124303021246D302124413001
:0C0D200021240024851E4D2E662E0800A4
:100E0000820700340E341134113411340A341B3487
:100E10000034003400341234123412341E341134CD
:100E2000103400340E341F341F341F341F341F3469
:100E3000003400340E3411341F341F341F341F3477
:100E4000003400340E34113411341F341F341F3475
:100E5000003400340E341134113411341F341F3473
:100E6000003400340E3411341134113411341F3471
:020E700000344C
:101000008617EB01EC01831607309F0083128701DE
:101010008715071587149D26AC26A226AC269D268B
:1010200020306B2656306B2647306B2641306B26BE
:101030003E306B26A22636306B2634306B2630309D
:101040006B262A306B2634306B2638306B263030D6
:101050006B26E124803086004B2186151D30C200AE
:10106000EF30C300C400EC0F3E28EB0A32306B02B5
:10107000031933214C214B21000041284B214C21E5
:101080004C2186114B218615502100000000C20B17
:101090004128C03086004B21861550210A30C500FA
:1010A00000000000000086114B218615CF3086001D
:1010B0000000CB3086000000CE3086000000CA3031
:1010C00086000000CD3086000000C9308600000098
:1010D000CC3086000000C8308600C30B53280000C7
:1010E00086114B218615CF3086000000CB3086005C
:1010F0000000CE3086000000CA3086000000CD30EF
:1011000086000000C93086000000CC308600000058
:10111000C8308600C40B7028000086114B2186154C
:101120005021851EA128C50B8D28000086110000C6
:101130000000000086155021051D56290000803052
:101140002B288617EB01EC019D26AC26A226AC26A7
:101150009D2620306B2656306B2647306B2641305B
:101160006B2631306B2632306B2638306B263030B0
:101170006B26A2262A306B2631306B2630306B2648
:1011800032306B2634306B26E124803086004630C6
:10119000C2008615EC0FD228EB0A32306B0203191D
:1011A0003321D5284B2100000000F030C300C400DB
:1011B00086110000000086154C2100000000C20BC3
:1011C000D828C03086000000000086154C210A3067
:1011D000C5000000C830860086110000CA308615A0
:1011E00086004B2100000000C830C30BEB28000034
:1011F000860086110000C930861586004B21F0302C
:10120000C300C830C40BF828000086008611000017
:10121000CC30861586004B21F030C400C830C30B9B
:1012200005290000860086110000C9308615860059
:101230004B2100000000C830C40B122900008600BA
:1012400086110000000086154C21851E0028C50B64
:101250002029000086110000000086154C21051D84
:1012600056298030C6289D26AC26A226AC269D266F
:1012700020306B2650306B2657306B2652306B2651
:101280005F306B266F306B2666306B2666306B26C0
:10129000861348290800080000000000000008002C
:1012A0000530BE00BE0B522900000800EB01EC0126
:1012B00086179D26AC26A226AC269D2620306B26BE
:1012C0004C306B268324E124D701831607309F001E
:1012D0000130870083128B130630900010108715A1
:1012E00007158710EC0F7929EB0A03306B020319FD
:1012F000332105197C29202B851D7F29532A0B2496
:101300000130210203188F298330200203188F290E
:101310009D26AC26A226AC269D268E247229EB01A2
:10132000EC012108A5002008A4000E25A701A601B4
:101330000330A500E830A40025252108C7002008B7
:10134000C600051AA729E124051AA72921240F3070
:10135000A3001930A2000D30A1002030A000A70189
:10136000A60124306024A50025306024A400252592
:10137000A701A6010330A500E830A4000E25A701AF
:10138000A6014708A5004608A40025252108C90094
:101390002008C8004B1CD229A701A601A501643072
:1013A000A4000E25A701A60128306024A50029303D
:1013B0006024A4009D26AC26A226AC269D262030C3
:1013C0006B2601252C1CE6292D306B26B625013015
:1013D0002D020318382A01302E020318382A013052
:1013E0002F0203181F2A013030020318222A01306D
:1013F00031020318252A013032020318042A013071
:1014000033020318072A0A2A3208303E6B263308B3
:10141000303E6B263408303E6B262C306B26350868
:10142000303E6B263608303E6B2620306B26A226D7
:1014300075306B266B306B2648306B2672292F086F
:10144000303E6B263008303E6B263108303E6B262E
:101450002E306B263208303E6B263308303E6B262A
:1014600020306B26A2266D306B2648306B26722901
:101470002D08303E6B262E08303E6B262C306B2616
:101480002F08303E6B263008303E6B263108203066
:101490006B26A22648306B2665306B266E306B2695
:1014A00020306B267229EB01EC0186179D26AC26B5
:1014B000A226AC269D2620306B2643306B26832443
:1014C000E124D701EC0F692AEB0A03306B02031900
:1014D000332185196C2A562905196F2A202B0B24D4
:1014E0000230210203187F2AFE30200203187F2ACF
:1014F0009D26AC26A226AC269D269B24622A210886
:10150000A5002008A4000E25A701A6010330A50010
:10151000E830A40025252108A5002008A4000F30EC
:10152000A3001930A2000D30A1002030A000252515
:10153000051AAB2AE124051AAB2A9D26AA24A22665
:10154000AC262108BD002C306B242008BD002D30B6
:101550006B24E124A7264B1CB32AA701A601A501F1
:101560006430A4000E252C306024A5002D306024AA
:10157000A400A701A6019D26AC26A226AC269D2686
:1015800020306B2601252C1CC72A2D306B26B62552
:1015900001302F0203180C2B013030020318F62AF9
:1015A000013031020318F92A013032020318DD2A12
:1015B000013033020318E02AE32A3208303E6B265A
:1015C0003308303E6B263408303E6B263508303EFB
:1015D0006B262C306B263608303E6B26A226203038
:1015E0006B2670306B2646306B26622A3008303E00
:1015F0006B263108303E6B263208303E6B262E308B
:101600006B263308303E6B2620306B26A2266E30C8
:101610006B2646306B26622A2F08303E6B262C3014
:101620006B263008303E6B263108303E6B26320880
:1016300020306B26A22602306B2646306B26622AAB
:10164000EB01EC0186179D26AC26A226AC269D2632
:1016500020306B2646306B268324E124051D2E2B7B
:10166000871507118714EC0F362B33210519502BE2
:101670009D26AC26A226AC269D2620306B26453022
:101680006B2653306B2652306B2620306B263E3053
:101690006B26E124831684309F0083128A114D2823
:1016A00061239D26AC26A226AC26B6259D26203099
:1016B0006B2646306B2678306B263E306B269523A2
:1016C000332B06309000E530C1000430BD00A0018E
:1016D000A101A201A3018F018E010C10101448304A
:1016E000BE000230BF00BE0B732BBF0B732B0C1C54
:1016F0007F2BA20A0319A30A0C100000852B0000FF
:1017000000000000000000000000C10B6F2BBD0BAB
:101710006F2B000010100C1C902BA20A0319A30AB7
:101720000F08A1000E08A000080001302F020318C6
:10173000A62B013030020318AB2B01303102031805
:10174000B02B013032020318B72BBC2B8230862617
:101750002F08303E6B26833086263008303E6B26BD
:101760008430862620306B263108303E6B2686304A
:1017700086263208303E6B26873086263308303E78
:101780006B26A22620306B263408303E6B263508A7
:10179000303E6B263608303E6B2620306B264830B4
:1017A0006B267A306B26080026309000C830C100C6
:1017B0000230BD00A001A101A201A3018F018E0191
:1017C0000C1010141E30BE000230BF00BE0BE62B02
:1017D000BF0BE62B0C1CF12BA20A0319A30A0C1059
:1017E000F62B00000000000000000000C10BE22BFF
:1017F000BD0BE22BB330BE00BE0BFC2B0000000083
:1018000010100C1C062CA20A0319A30A0F08A10031
:101810000E08A0000800D423013022020318172C60
:101820001F3021020318172C0130CB001E2CCB01D6
:10183000A701A601A5010A30A4002525A701A6013C
:1018400008009D26AA240F30A3001930A2000D30F5
:10185000A1002030A000A701A6014708A500460866
:10186000A4002525A701A601A5010A30A40025256D
:101870002108BD0024306B242008BD0025306B24D6
:10188000B625A22643306B2678306B2620306B2697
:101890003408303E6B263508303E6B263608303E25
:1018A0006B2670306B2646306B264808BD00293009
:1018B0006B244908BD0028306B24E124A7260800CA
:1018C000031783128D0083168C130C1483120C08DB
:1018D000031383120800031783168C186D2C8312D0
:1018E0008D00031383123D0803178C0083168C139D
:1018F0000C158B1355308D00AA308D008C140C11F3
:1019000003138312080020306B264D306B266530A0
:101910006B2674306B2672306B26080020306B26E5
:101920004C306B2678306B262D306B262D306B2695
:101930002D306B26080020306B2643306B26783024
:101940006B2620306B2645306B2652306B2652308A
:101950006B26080020306B2643306B2661306B26E7
:101960006C306B2669306B2662306B2672306B26CA
:101970002E306B26080020306B2653306B266130EA
:101980006B2676306B2620306B2645306B26453033
:101990006B2608009730BE000330BF00BE0BCE2C74
:1019A000BF0BCE2C0800AC30BE001330BF00063099
:1019B000C000BE0BD92CBF0BD92CC00BD92C0000FA
:1019C00008005430BE008A30BF000330C000BE0B98
:1019D000E72CBF0BE72CC00BE72C00000800A4018C
:1019E000A501A601A7010800A001A101A201A30170
:1019F000A401A501A601A701A801A901AA01AB01A3
:101A0000080028260318080023082706B700F12538
:101A1000031027082306B71F803E0800B7011226CF
:101A2000031C25260318080000260D261F30B800C9
:101A300038262B0D0318F125031C230D031808006D
:101A4000B80B182D371815260800B70124082504EF
:101A500026042704003C031C1226031C2526031819
:101A60000800A801A901AA01AB0138261F30B8005F
:101A7000382627082B02031D472D26082A02031D9E
:101A8000472D25082902031D472D24082802031C81
:101A9000592D2408A8022508031C250FA902260891
:101AA000031C260FAA022708031C270FAB020310F2
:101AB0002014B80B382D371815260800B701122648
:101AC00003103C2627082B02031D702D26082A022E
:101AD000031D472D25082902031D702D2408280207
:101AE000031C7B2DA00F7B2DA10F7B2DA20F7B2D27
:101AF000A30A03190800371815260800230D031838
:101B00000800002609261030B800A80DA90DAA0D5E
:101B1000AB0DA40DA50DA60DA80DA90DAA0DAB0D1D
:101B2000A40DA50DA60D0314A00DA10DA20D220854
:101B30002602031DA12D21082502031DA12D200829
:101B40002402031CAE2D2008A4022108031C210F2F
:101B5000A5022208031C220FA602A0142010B80B15
:101B6000852D0310A20CA10CA00C0800B7011226B1
:101B70000318080041262030B800A00DA10DA20DC9
:101B8000A30D363084000A30B900800D0A300002FF
:101B9000031880008403B90BC52DB80BBD2D371871
:101BA0002C1403100800B7002030B8002C3084003B
:101BB0003708B9000A300310840A03188007800C24
:101BC000B90BDC2DA30CA20CA10CA00CB80BD62DCC
:101BD0000008FF3E031C230D031808002C181526CF
:101BE00008002408A00725080318250FA1072608C8
:101BF0000318260FA20727080318270FA3070800BA
:101C00002008A8002108A9002208AA002308AB0088
:101C10000800A401A501A601A701A001A101A2013C
:101C2000A3010800230D031C080023088039A00924
:101C3000A109A209A309A00F222EA10F222EA20FF3
:101C4000222EA30AB70A23070800270D031C080049
:101C500027088039A409A509A609A709A40F352ECC
:101C6000A50F352EA60F352EA70AB70A270708009D
:101C7000A00DA10DA20DA30DA80DA90DAA0DAB0DD0
:101C80000800AC01AD01AE01AF01B001B101B2017C
:101C9000B301B401B501B6010800B326B326B326DB
:101CA0000330C20086008616000000000000861285
:101CB000B326C20B532E02308600861600000000A9
:101CC000000086128601BC26283086260C30862627
:101CD000063086260800BD003D0E0F3910388604F8
:101CE000E0388605861600000000000086123D08D8
:101CF0000F3910388604E03886058616000000008B
:101D0000000086121F308604BC260800BD003D0E70
:101D10000F398604E03886058616000000000000B2
:101D200086123D080F398604E038860586160000C5
:101D3000000000008612BC260800803086260C3089
:101D400086260800C03086260C3086260800013022
:101D500086260C30862608001030C20020306B2604
:101D6000C20BAE2E08002F30BE000630BF00BE0BE7
:101D7000B72EBF0BB72E08004130BE00BE0BBE2EE3
:021D8000080059
:02400E00713F00
:104200007F0000007F0000007F0000000000000031
:1042100003000000000000007F000000000000001C
:1042200064000000000000006400000000000000C6
:10423000000000000000000000000000000000007E
:10424000000000000000000002008A0000000000E2
:1042500027001000000000001900640000000000AA
:00000001FF
